:100000000C9446000C9466000C9466000C946600F8
:100010000C9466000C9466000C9466000C946600C8
:100020000C9466000C946F000C9466000C946600AF
:100030000C9466000C9466000C9466000C946600A8
:100040000C9466000C9466000C9466000C94660098
:100050000C9466000C9466000C9466000C94660088
:100060000C9466000C9466000C9466000C94660078
:100070000C9466000C9466000C9466000C94660068
:100080000C9466000C94E5020C94660011241FBECB
:10009000CFEFD0E1DEBFCDBF11E0A0E0B1E0E4EDF5
:1000A000FAE000E00BBF02C007900D92A030B1074C
:1000B000D9F71BBE11E0A0E0B1E001C01D92A23F44
:1000C000B107E1F70E948B000C9468050C940000C6
:1000D0008BE085BD89EF83BD80E887BF08951F92BF
:1000E0000F920FB60F9211248F939F93809100016E
:1000F00090910101019690930101809300019F91DD
:100100008F910F900FBE0F901F90189585B390E3BD
:10011000892785BB0895EF92FF920F931F938FEF6E
:1001200084BB85B390E3892785BBF8948DE08093E9
:10013000F10180E090E060E070E00E94C2020E9465
:10014000B0020E94680080E090E060E070E00E94F1
:100150003E0586E890E060E070E040E050E021E09D
:1001600030E004EF11E0E2E3EE2EF12C0E94F80003
:100170008DE495E060E070E040E050E021E030E0A8
:100180000AE010E0EE24FF240E94F80078940E9418
:10019000CA01FDCFFC01838994898230910539F52C
:1001A0008281882319F0813011F511C0838181305B
:1001B00039F480E090E060E070E00E94500508951E
:1001C00080E090E060E070E00E9447050895838140
:1001D000813039F480E090E060E070E00E944905F1
:1001E000089580E090E060E070E00E944B05089583
:1001F000EF92FF920F931F93CF93DF93E0E0F0E035
:10020000AE2FEF01B4E0CC0FDD1FBA95E1F7CE1BA6
:10021000DF0BCE5FDE4FBD85BB2329F0AF5F31968C
:10022000EC30F10569F7B0E0FD01E295F295F07F61
:10023000FE27E07FFE27EA1BFB0BEE5FFE4F91835C
:100240008083738362835583448337832683E114D9
:10025000F10411F4168608C082E3E816F10411F4E3
:1002600081E001C082E08687FD0134E0EE0FFF1FD0
:100270003A95E1F7EA1BFB0BEE5FFE4F8685C82F30
:10028000D0E0CA54DE4F8881E80EE4868F5F888311
:100290001187008781E08587F89480910001909113
:1002A0000101800F911FFD0124E0EE0FFF1F2A9531
:1002B000E1F7EA1BFB0BEE5FFE4F93878287789492
:1002C000DF91CF911F910F91FF90EF900895DF92F2
:1002D000EF92FF920F931F93E0E0F0E0DE2EDF013C
:1002E000A295B295B07FBA27A07FBA27AE1BBF0BED
:1002F000AE5FBE4F1D96AC91AA2329F0D3943196E0
:10030000EC30F10559F7AD2DB0E0FD01E295F29525
:10031000F07FFE27E07FFE27EA1BFB0BEE5FFE4F20
:1003200091838083738362835583448337832683D9
:10033000E114F10411F4168608C082E3E816F10412
:1003400011F481E001C082E08687FD0184E0EE0FB8
:10035000FF1F8A95E1F7EA1BFB0BEE5FFE4FA685B8
:10036000B0E0AA54BE4F8C91E80EE4868F5F8C9368
:100370001187008781E085878091000190910101BC
:10038000800F911F938782871F910F91FF90EF90AD
:10039000DF900895CF93DF93F894609100017091FE
:1003A000010178941092B9018091BC018F5F809314
:1003B000BC018091BC01883C49F48091BB018695C9
:1003C0008093BA011092BB011092BC0180E090E0D2
:1003D0004FEF2FEFFC0134E0EE0FFF1F3A95E1F7EE
:1003E000E81BF90BEE5FFE4F3585332379F0309132
:1003F000B9013F5F3093B901A285B3856A177B07C6
:1004000028F03485341710F44485282F01968C3059
:10041000910501F72F3F71F18091BB018F5F8093B0
:10042000BB01332727FD3095E90184E0CC0FDD1FA8
:100430008A95E1F7C21BD30BCE5FDE4FE881F981CD
:100440008A819B816C817D8109958E819F81009736
:1004500049F41D86EE85F0E0EA54FE4F808181501C
:10046000808308C02A853B8588859985820F931FE4
:100470009B878A8781E0DF91CF91089520E030E06B
:10048000F90154E0EE0FFF1F5A95E1F7E21BF30B61
:10049000EE5FFE4F4081518148175907C1F44585F1
:1004A0004423A9F0F8948091000190910101860FF6
:1004B000971FF90144E0EE0FFF1F4A95E1F7E21B99
:1004C000F30BEE5FFE4F93878287789408952F5F3A
:1004D0003F4F2C303105A1F6089520E030E0F901BE
:1004E000A4E0EE0FFF1FAA95E1F7E21BF30BEE5F0E
:1004F000FE4F408151814817590761F445854423D7
:1005000049F08091000190910101860F971F938718
:10051000828708952F5F3F4F2C30310501F70895F2
:1005200020E030E0F901B4E0EE0FFF1FBA95E1F7EB
:10053000E21BF30BEE5FFE4F4081518148175907D4
:1005400049F41586E685F0E0EA54FE4F808181503B
:10055000808308952F5F3F4F2C30310519F70895A0
:1005600080E090E0FC0124E0EE0FFF1F2A95E1F708
:10057000E81BF90BEE5FFE4F158601968C30910556
:1005800089F708958091F101880F8160809372004E
:1005900080E480937000E1E7F0E080818C7F8083CD
:1005A0008FEF8093730095EC9093740021E030E01E
:1005B0003093C0012093BF011092BE018093EB01E4
:1005C0001092D5011092D40108951F920F920FB688
:1005D0000F920BB60F921124EF92FF920F931F937D
:1005E0002F933F934F935F936F937F938F939F933B
:1005F000AF93BF93EF93FF938091BF019091C001A0
:10060000817C09F4BFC08091710090E0887F907078
:100610008036910509F49CC08836910509F480C0A4
:100620008037910509F494C08837910509F478C0A2
:100630008038910581F08838910509F499C0803996
:10064000910549F08839910509F492C0803A9105E5
:1006500009F096C093C08091BF019091C001803491
:10066000910581F4809173008093C2018FEF809394
:10067000EB0180E890E09093C0018093BF0110925D
:10068000BE017CC08091BF019091C001803891056E
:1006900009F074C09091BE018091C2019817A0F436
:1006A0008091BE01E82FF0E090917300EF53FE4F70
:1006B00092838F5F8093BE019091EB0180917300D4
:1006C00089278093EB015AC08091BE01803111F5DA
:1006D000809173008093D3019091EB018091D301BD
:1006E000981719F081E090E002C082E090E09093CA
:1006F000D5018093D4018AEC90E061EC71E040E098
:1007000050E020E030E000E010E0EE24FF240E9402
:1007100067012EC08091BE018F5F8093BE012EC005
:100720008091EF018F5F8093EF018091EC018A301F
:1007300078F487EA94E060E070E040E050E020E088
:1007400030E002E310E0A2E3EA2EF12C0E94670100
:10075000809173008093C1011092D5011092D40151
:100760001092BE0185EC8093740080E490E076C026
:1007700081E090E09093C0018093BF0185ECCEC0F2
:1007800085E4CCC08091710090E0887F90708830C3
:100790009105B1F08031910599F088319105D1F042
:1007A0008032910509F48CC088329105D1F08033F4
:1007B000910509F458C08833910509F0A8C059C0C3
:1007C0008091D6018093730085E88093740088E05F
:1007D00090E044C01092BD018091D70180937300D6
:1007E00038C08091BD018131D9F485E980937400CE
:1007F00080E290E09093C0018093BF011092EC01E1
:100800008091ED019091EE0101969093EE0180931D
:10081000ED0182EC92E060E070E00E946D0280C029
:100820009091BD018091D701981738F08091E8012F
:10083000809373008091BD0109C08091BD01E82FB4
:10084000F0E0EA52FE4F9281909373008F5F8093A5
:10085000BD0185E88093740080E190E09093C00131
:100860008093BF015DC08091EF018F5F8093EF01A6
:100870002CC08091EF018F5F8093EF0182EC92E0BA
:1008800060E070E00E946D028091EC018A3080F49B
:1008900087EA94E060E070E040E050E020E030E083
:1008A00002E310E0F2E3EF2EF12C0E94670106C094
:1008B00088E290E09093C0018093BF0185E82EC04C
:1008C0008091F0018F5F8093F00182EC92E060E014
:1008D00070E00E946D028091EC018A3080F487EA1A
:1008E00094E060E070E040E050E020E030E002E3BF
:1008F00010E0E2E3EE2EF12C0E94670106C088E2D0
:1009000090E09093C0018093BF0185E907C084E027
:1009100090E09093C0018093BF0185E080937400C4
:10092000FF91EF91BF91AF919F918F917F916F91C7
:100930005F914F913F912F911F910F91FF90EF90F9
:100940000F900BBE0F900FBE0F901F901895EF9257
:10095000FF920F931F938091BF019091C00181304E
:10096000910559F087EA94E060E070E040E050E0E3
:1009700020E030E005E010E01AC01092BD0185EAE9
:100980008093740082E090E09093C0018093BF0157
:100990008091EC018F5F8093EC0182EC92E060E04B
:1009A00070E040E050E020E030E000E117E2B2E328
:1009B000EB2EF12C0E94F8001F910F91FF90EF9009
:1009C0000895EF92FF920F931F939091EC0199235A
:1009D00009F44AC09091EC019A3009F445C081E0D5
:1009E0003EC09FEF9093E801E62FF72F20E030E024
:1009F0000FC09081D901AA52BE4F12969C931297B4
:100A00009091E801519195279093E8012F5F3F4F16
:100A1000241778F391E09093EC0190E0880F991FF0
:100A20008093D6014093D7011092BD0185EA80934F
:100A3000740082E090E09093C0018093BF0182EC4B
:100A400092E060E070E040E050E020E030E005E05F
:100A500010E0E2E3EE2EF12C0E94F80080E01F91FE
:100A60000F91FF90EF9008952091BF013091C00148
:100A70002130310509F4B5CF82E0F1CF84B3836032
:100A800084BB85B38C7F85BBD098D8980895A898EF
:100A90000895A99A0895A9980895C899A8980895BD
:100AA000EF92FF920F931F93A89A87E495E060E07E
:100AB00070E040E050E020E030E000E61AEEEE2486
:100AC000FF240E94F8001F910F91FF90EF9008956E
:040AD000F894FFCFC8
:00000001FF
